:1000000010308A00232B0000FF00030E8301A100A3
:100010000A08A0008A010408A2007708A300780853
:10002000A4007908A5007A08A6007B08A70083131E
:1000300083128B1D1D280B1840288C308400801ED5
:1000400023288C1A43288C308400801C29288C1883
:1000500046288B1E2D280B194928220884002308C6
:10006000F7002408F8002508F9002608FA002708F8
:10007000FB0020088A00210E8300FF0E7F0E09007E
:100080008A110A1218298A150A1200288A110A12DE
:100090005D2B8A110A1240290A108A100A11820760
:1000A000483465346D3469344F3453342034563415
:1000B0002534733420342C3420344B342D345434D0
:1000C000653461346D34203453342E3441342E344D
:1000D00020342834203441346C346534783461342D
:1000E0006E34643472346534203443346F346C3489
:1000F0006F347434203429342034203400340A100E
:100100008A100A11820731342E34343430340034EA
:100110000A108A100A118207333431342D346A34BC
:10012000753469346C342E342D3430343334003427
:100130000A108A100A118207313436343A343234C4
:1001400033343A343534363400340A108A100A1104
:10015000820745342D344D34613469346C34203495
:100160003A34203469346E3466346F344034683441
:1001700065346D346934733473346F346E342E34B3
:1001800063346F346D340D340A340D340A34003462
:100190000A108A100A11820762342C3448346534FC
:1001A0006D3469344F3453345F3476345F342534DE
:1001B00073340D340A3400340A108A100A1182078D
:1001C00055346E346B346E346F3477346E3420347F
:1001D00043346F346D346D3461346E3464342034A0
:1001E0003F3421340D340A3400340A108A100A11C5
:1001F000FC3E03188A0A82004434E9346D346134C9
:1002000072347234613467346534203465346E344A
:1002100020346D346F3464346534203449346E34A2
:100220007434653472346E3465340D340A340034F9
:100230000030AD180130013C031D3C29F930F700B6
:10024000F70B2029000000000030061A0130003AA8
:10025000031D3C29C6012D13061E2D17C60A8B113E
:100260001030F80006389200BB30831692008312DB
:10027000910183168C1483120B108A110A122D28F7
:10028000AA1B52292A080F3C2C07F700F71B4F29FD
:1002900077080E3C03184F290810881051290814BC
:1002A000881062292A08003C0F3C2C07F700F71B36
:1002B000602977080E3C031860290810881062290D
:1002C00008108814AB1B74292B080F3C2C07F7006F
:1002D000F71B712977080E3C031871290811881142
:1002E00073290815881184292B08003C0F3C2C0722
:1002F000F700F71B822977080E3C031882290811A2
:100300008811842908118815AC0A2C080F3C0318A1
:100310008A29AC015C08F700013077020319B5297E
:10032000033077020319DF290A3077020319FF2906
:100330000C30770203193A2A0F30770203196C2A1E
:10034000143077020319712A163077020319AC2A88
:10035000193077020319DF2A233077020319002BA3
:10036000C83077020319052B0D2B00302D180130F2
:10037000013C031DDE293030F8001F08C73978041E
:100380009F001330F700F70BC329000000001F1572
:100390001F19C8291E08CE003830F8001F08C739B9
:1003A00078049F001330F700F70BD42900000000F9
:1003B0001F151F19D9291E08CF0086140D2B0030D8
:1003C0002D180130013C031DFE291F151F19E629B8
:1003D0001E084F02D7003030F8001F08C7397804D4
:1003E0009F001330F700F70BF329000000001F15E2
:1003F0001F19F8291E084F02D60086100D2B003059
:100400002D180130013C031D392A0830F8001F085F
:10041000C73978049F001330F700F70B0D2A00004E
:1004200000001F151F19122A1E08C9000030F8000D
:100430001F08C73978049F001330F700F70B1E2AF6
:10044000000000001F151F19232A1E08C8001030C5
:10045000F8001F08C73978049F001330F700F70B26
:100460002F2A000000001F151F19342A1E08CA0079
:1004700006150D2B00302D180130013C031D6B2A91
:100480001F151F19412A1E084A02D2000830F80021
:100490001F08C73978049F001330F700F70B4E2A66
:1004A000000000001F151F19532A1E084902D10021
:1004B0000030F8001F08C73978049F001330F70098
:1004C000F70B602A000000001F151F19652A1E087F
:1004D0004802D00006110D2BDD08031D702A881775
:1004E0000D2B00302D180130013C031DAB2A2030AC
:1004F000F8001F08C73978049F001330F700F70B86
:100500007F2A000000001F151F19842A1E08CC0036
:100510002830F8001F08C73978049F001330F7000F
:10052000F70B902A000000001F151F19952A1E08BE
:10053000CD001830F8001F08C73978049F00133029
:10054000F700F70BA12A000000001F151F19A62AAB
:100550001E08CB0086150D2B00302D180130013CF4
:10056000031DDE2A1F151F19B32A1E084B02D300D4
:100570002030F8001F08C73978049F001330F700B7
:10058000F70BC02A000000001F151F19C52A1E08FE
:100590004C02D4002830F8001F08C73978049F00A7
:1005A0001330F700F70BD22A000000001F151F19A7
:1005B000D72A1E084D02D50086112D160D2B2914A1
:1005C0002908831687008312D801071CD80AA914AA
:1005D0002908831687008312D901871CD90A291597
:1005E0002908831687008312DA01071DDA0AA91683
:1005F0002908831687008312DB01871EDB0A0D2B77
:10060000DD08031D042B88130D2BDC01DD0A5D08BA
:100610000A3C03180C2BDD010D2BDC0A0B118A118F
:100620000A122D2801304502EF3E0318452B113EDA
:10063000482B0530AA000A30AB00452B0A30AA002F
:10064000AB00452B0A30AA000530AB00452BF63035
:10065000AA000A30AB00452BAA01AB01452B0A309A
:10066000AA00F630AB00452BFB30AA00F630AB00F9
:10067000452BF630AA00AB00452BF630AA00FB3024
:10068000AB00452B452B452B452B8A110A122D2CEF
:100690000A148A140A118207192B1E2B222B272BCE
:1006A0002C2B2F2B342B392B3D2B452B452B422B21
:1006B000452B452B452B432B442B01304602F33E63
:1006C0000318382C0D3E3D2CAD13061EAD1700301F
:1006D000AD1B0130013C0319762B1030F80092005D
:1006E000BB30831692008C1083128B15382C43106C
:1006F000061E4314382CC310061EC3140030C31842
:100700000130003A03198D2B1030F8009200BB30F5
:10071000831692008C1083128B15382C4311061E01
:100720004315003043190130003A0319A02B103053
:10073000F8009200BB30831692008C1083128B1548
:10074000382CC311061EC3150030C3190130003AFE
:100750000319B32B1030F8009200BB3083169200BF
:100760008C1083128B15382C4312061E4316003052
:10077000431A0130003A0319C62B1030F8009200DA
:10078000BB30831692008C1083128B15382CC31249
:10079000061EC316382C4313061E4317382CC313EA
:1007A000061EC317382C4410061E4414382CC410DF
:1007B000061EC414382C4411061E4415382CC411CE
:1007C000061EC4150030431B0130F700770E831658
:1007D000B000B00DE030B00500308312C31B013013
:1007E000F700F70EF030F705770883163004B200F3
:1007F0000030831244180130F700F70DF70DF70DA4
:10080000F830F705770883163204B40000308312FD
:10081000C4180130F700F70DF70DFC30F705770825
:1008200083163404B6000030831244190130F700F7
:100830000310F70D770883163604B80000308312D2
:10084000C4190130831638048312C5000030AD1975
:100850000130013C031D2D2C122BAD161030F80079
:100860009200BB30831692008C1083128B15382CAB
:10087000C60A8C108A110A122D280A108A100A152D
:100880008207642B772B7B2B8E2BA12BB42BC72BB2
:10089000CB2BCF2BD32BD72BDB2BDF2B83163F0878
:1008A000F8013E020318572C3E08F700632CF701AD
:1008B0000830C000BE0DF70D3F0877020318F7009F
:1008C000F80DC00B5A2C8312003483163C08F70035
:1008D000BC1B6E2C3D1D7D2C2030732CF709F70AB4
:1008E0007708BC002D30F80083120C1A792C83167F
:1008F000742C990083163D1DBD153C08BE00643064
:10090000BF0083124E2477088316BC00780830306D
:10091000031D912C3D189C2CBD199C2C3D1A203098
:10092000932CBD113D12F807780883120C1A9A2CEB
:100930008316952C990083163C08BE000A30BF0030
:1009400083124E2477088316BC0078083030031DCC
:10095000AD2CBD19B62C3D1A2030F807780883124B
:100960000C1AB42C8316AF2C990083163030BC07B8
:100970003C0883120C1ABE2C8316B92C9900003443
:10098000780883163C08BE006430BF0083124E24F2
:1009900077088316BC0078083030031DD62C3D182C
:1009A000E12CBD19E12C3D1A2030D82CBD113D128F
:1009B000F807780883120C1ADF2C8316DA2C9900BA
:1009C00083163C08BE000A30BF0083124E2477080D
:1009D0008316BC0078083030031DF22CBD19FB2CA7
:1009E0003D1A2030F807780883120C1AF92C831668
:1009F000F42C990083163030BC073C0883120C1A83
:100A0000032D8316FE2C9900003483163D08413CCB
:100A100003180F2D41303D020A3EBE00122D30302A
:100A20003D02BE003E08F8008312003494138C117E
:100A300083163D08831293000230941B262D8C1DD3
:100A40001F2D00308316111B01308312F800003473
:100A50008316911591192A2D77189112771C9116EA
:100A60001116111A312D83121308F8000034AA014F
:100A7000AB01C801C901CA01CB01CC01CD01CE0136
:100A8000CF01D001D101D201D301D401D501D601CA
:100A9000D701D801D901DA01DB0183169F01831246
:100AA0001F083839C1389F0083160912F701F71D56
:100AB000642D073083128101813084008313000884
:100AC000C0390F388000831664008130840000082C
:100AD000C03977048000831290010030F800920042
:100AE0000030831692008312291529088316870087
:100AF000831297019701A91429088316870083128E
:100B00009D019D012F308316850030308600003016
:100B10008800091489140915103083128500860194
:100B20008801890183168117F80083129200BB3077
:100B3000831692008312910183160108C03901388F
:100B4000810083128101B53090008F018E01EC018C
:100B50006C084C20EC0AF70077080C1EAD2D9900AC
:100B600008306C02031DA82DED016D087F200038B0
:100B70000319BF2DED0A0C1EBB2D9900B52D0A30AF
:100B8000EE006E084C20EE0AF70077080C1EC62D0A
:100B900099002E306E02031DC12DEC016C088820D7
:100BA000EC0AF70077080C1ED32D99000B306C026D
:100BB000031DCE2D20300C1EDB2D990040300C1E65
:100BC000DF2D990020300C1EE32D9900EC016C08FC
:100BD0009820EC0AF70077080C1EEC2D99000830DD
:100BE0006C02031DE72D0D300C1EF42D99000A3008
:100BF0000C1EF82D9900EC016C08A520EC0AF700FA
:100C000077080C1E012E99001E306C02031DFC2D6E
:100C10008B168B1500302D190130013C031D132E4E
:100C200083168C168312C0308B048A110A16682B27
:100C30008316A308031D202E83122D10222E831647
:100C400083122D1400348316A308031D2B2E831248
:100C5000AD102D2E83168312AD1400348316A30815
:100C6000031D362E83122D11382E831683122D1557
:100C700000348316A308031D412E8312AD11432EA9
:100C800083168312AD150034A63084008313000848
:100C900003194F2E4D2E00000000800B4B2E003408
:100CA000A5308400831300080319632E0630F80072
:100CB000F701F70B592EF80B582E7B30F700F70B86
:100CC0005F2E800B562E003483162308A4002408C0
:100CD000F700F70883120319762E01307702031903
:100CE000E12E0230770203194C2F932F0830F800C1
:100CF0001F08C73978049F001330F700F70B7E2ECA
:100D0000000000001F151F19832E1E08C9000030A7
:100D1000F8001F08C73978049F001330F700F70B5D
:100D20008F2E000000001F151F19942E1E08C800EA
:100D30001030F8001F08C73978049F001330F700FF
:100D4000F70BA02E000000001F151F19A52E1E086E
:100D5000CA00061502308316A5009330A600831240
:100D600044268316A50BAD2E83121F151F19B62E10
:100D70001E084A02D2000830F8001F08C73978045C
:100D80009F001330F700F70BC32E000000001F1563
:100D90001F19C82E1E084902D1000030F8001F0894
:100DA000C73978049F001330F700F70BD52E0000E9
:100DB00000001F151F19DA2E1E084802D000061168
:100DC000932F2030F8001F08C73978049F00133094
:100DD000F700F70BE92E000000001F151F19EE2E7B
:100DE0001E08CC002830F8001F08C73978049F007F
:100DF0001330F700F70BFA2E000000001F151F1923
:100E0000FF2E1E08CD001830F8001F08C7397804DF
:100E10009F001330F700F70B0B2F000000001F1589
:100E20001F19102F1E08CB00861502308316A5004F
:100E30009330A600831244268316A50B182F831225
:100E40001F151F19212F1E084B02D3002030F80058
:100E50001F08C73978049F001330F700F70B2E2FB7
:100E6000000000001F151F19332F1E084C02D4006C
:100E70002830F8001F08C73978049F001330F700A6
:100E8000F70B402F000000001F151F19452F1E08EB
:100E90004D02D5008611932F3030F8001F08C73956
:100EA00078049F001330F700F70B542F0000000068
:100EB0001F151F19592F1E08CE003830F8001F08C3
:100EC000C73978049F001330F700F70B652F000037
:100ED00000001F151F196A2F1E08CF00861402304C
:100EE0008316A5009330A600831244268316A50B13
:100EF000722F83121F151F197B2F1E084F02D70058
:100F00003030F8001F08C73978049F001330F7000D
:100F1000F70B882F000000001F151F198D2F1E08CA
:100F20004F02D600861005308316A5008312502686
:100F30000034503083162307840083130008F80020
:100F4000831200348316A308031DAA2F83120812EC
:100F5000AC2F8316831208160034F701F8018316AC
:100F60002A0803102B18F707F70CF80CAB18F70733
:100F7000F70CF80C2B19F707F70CF80CAB19F7075F
:100F8000F70CF80C2B1AF707F70CF80CAB1AF7074D
:100F9000F70CF80C2B1BF707F70CF80CAB1BF7073B
:100FA000F70CF80C831200348316A308031DDC2F02
:100FB00083120813DE2F831683120817003483165A
:100FC000A3080319E72F83120512E92F8316831252
:100FD00005160034831623088312AA0083162408FA
:100FE0008312AB000034EC08031DF82F8812F92F90
:080FF00088168A110A16F02B85
:101000008316B901BA0183128C1E16282E304207AE
:10101000840083138C1E0A281A0880004208123CA0
:10102000031C1328C20A83160328831201304202CC
:101030002E3E8400831300080D3C031D332E2E0822
:10104000F7004230770203196A2844307702031907
:101050009C28453077020319CD28483077020319C0
:10106000F42849307702031909294C307702031913
:101070004A294D307702031977294E307702031938
:101080000E2A4F30770203197B2A5030770203195A
:10109000E82A5130770203197F2B52307702031967
:1010A000D82B533077020319A02C54307702031940
:1010B000E72C553077020319002D573077020319BA
:1010C000782D583077020319FF2D5A307702031913
:1010D0000C2E1B2E8316BC013C088A118312C820DB
:1010E0008A158316BC0AF70083120C1A7928831616
:1010F000742899000B3083163C02031D6C28BD0137
:101100003D088A1183127F208A150038031993281D
:101110008316BD0A83120C1A8F2883168A28990019
:101120008316802883120D300C1E942899000A30F3
:101130000C1E98289900322E30082D3C031DB12832
:1011400030303102003CAA0033082D3C031DAD288D
:1011500030303402003CAB00B02830303302AB00FA
:10116000C02830303002AA0032082D3C031DBD28B3
:1011700030303302003CAB00C02830303202AB00CC
:1011800064300C1EC12899000D300C1EC528990032
:101190000A300C1EC9289900322E65300C1ECE284C
:1011A00099002C300C1ED22899002A088316BC0006
:1011B0000130BD008A11831265248A152C300C1E63
:1011C000DF2899002B088316BC000130BD008A116E
:1011D000831265248A150D300C1EEC2899000A3004
:1011E0000C1EF0289900322E30303002003A031DD8
:1011F000FB280812FC28081668300C1EFD289900F0
:101200000D300C1E012999000A300C1E0529990089
:10121000322E69300C1E0A2999002C300C1E0E2922
:10122000990058088316BC001830BD008A1183123B
:1012300065248A152C300C1E1B2999005908831629
:10124000BC001830BD008A11831265248A152C3029
:101250000C1E282999005A088316BC001830BD00BE
:101260008A11831265248A152C300C1E35299900A9
:101270005B088316BC001830BD008A1183126524F8
:101280008A150D300C1E422999000A300C1E462981
:101290009900322E30303002003A031D5129881354
:1012A0005229881730303202003A031D592988121A
:1012B0005A29881630303402003A031D6129081378
:1012C0006229081730303602003A031969290512DD
:1012D0006A2905166C300C1E6B2999000D300C1E06
:1012E0006F2999000A300C1E73299900322E30089C
:1012F000F70030307702031986293130770203195D
:10130000B729323077020319E8290D2A6D300C1EF7
:10131000872999002C300C1E8B2999004A088316C6
:10132000BC00BD018A118312C0248A152C300C1E0A
:101330009729990048088316BC00BD018A118312C1
:10134000C0248A152C300C1EA32999004908831645
:10135000BC00BD018A118312C0248A150D300C1EF9
:10136000AF2999000A300C1EB32999000D2A6D305F
:101370000C1EB82999002C300C1EBC2999004D0870
:101380008316BC00BD018A118312C0248A152C303B
:101390000C1EC82999004C088316BC00BD018A1197
:1013A0008312C0248A152C300C1ED42999004B08B6
:1013B0008316BC00BD018A118312C0248A150D302A
:1013C0000C1EE02999000A300C1EE42999000D2A10
:1013D0006D300C1EE92999002C300C1EED29990066
:1013E0004F088316BC00BD018A118312C0248A15E0
:1013F0002C300C1EF92999004E088316BC00BD0143
:101400008A118312C0248A150D300C1E052A9900FA
:101410000A300C1E092A99000D2A322E6E300C1E3D
:101420000F2A99002C300C1E132A9900520883169B
:10143000BC00BD018A118312C0248A152C300C1EF9
:101440001F2A990050088316BC00BD018A1183121F
:10145000C0248A152C300C1E2B2A990051088316A3
:10146000BC00BD018A118312C0248A152C300C1EC9
:10147000372A990055088316BC00BD018A118312D2
:10148000C0248A152C300C1E432A99005408831658
:10149000BC00BD018A118312C0248A152C300C1E99
:1014A0004F2A990053088316BC00BD018A1183128C
:1014B000C0248A152C300C1E5B2A9900570883160D
:1014C000BC00BD018A118312C0248A152C300C1E69
:1014D000672A990056088316BC00BD018A11831241
:1014E000C0248A150D300C1E732A99000A300C1E78
:1014F000772A9900322E6F300C1E7C2A99002C30EE
:101500000C1E802A99004A088316BC00BD018A116E
:101510008312C0248A152C300C1E8C2A990048088E
:101520008316BC00BD018A118312C0248A152C3099
:101530000C1E982A990049088316BC00BD018A1127
:101540008312C0248A152C300C1EA42A99004D0841
:101550008316BC00BD018A118312C0248A152C3069
:101560000C1EB02A99004C088316BC00BD018A11DC
:101570008312C0248A152C300C1EBC2A99004B08FB
:101580008316BC00BD018A118312C0248A152C3039
:101590000C1EC82A99004F088316BC00BD018A1191
:1015A0008312C0248A152C300C1ED42A99004E08B0
:1015B0008316BC00BD018A118312C0248A150D3028
:1015C0000C1EE02A99000A300C1EE42A9900322EE3
:1015D0003008F700303077020319F72A31307702EC
:1015E0000319282B323077020319592B7E2B7030C8
:1015F0000C1EF82A99002C300C1EFC2A9900520867
:101600008316BC00BD018A118312C0248A152C30B8
:101610000C1E082B990050088316BC00BD018A11CE
:101620008312C0248A152C300C1E142B99005108EB
:101630008316BC00BD018A118312C0248A150D30A7
:101640000C1E202B99000A300C1E242B99007E2B97
:1016500070300C1E292B99002C300C1E2D2B99005C
:1016600055088316BC00BD018A118312C0248A1557
:101670002C300C1E392B990054088316BC00BD0178
:101680008A118312C0248A152C300C1E452B990018
:1016900053088316BC00BD018A118312C0248A1529
:1016A0000D300C1E512B99000A300C1E552B990041
:1016B0007E2B70300C1E5A2B99002C300C1E5E2B8A
:1016C000990057088316BC00BD018A118312C024FB
:1016D0008A152C300C1E6A2B990056088316BC0004
:1016E000BD018A118312C0248A150D300C1E762B81
:1016F00099000A300C1E7A2B99007E2B322E713005
:101700000C1E802B9900003064028316BC008312EB
:1017100065088316BD001830031C1930BD023D0852
:10172000BE0083120C1A962B8316912B9900003061
:1017300064028316BC00831265088316BD0018304E
:10174000031C1930BD023C08BE0083120C1AAA2BE0
:101750008316A52B9900DF015F08073C031CBF2BF4
:1017600050305F078400831300088316BC00831287
:101770000C1ABC2B8316B72B9900DF0AAC2BDF01A8
:101780005F08073C031CD32B48305F07840083139A
:1017900000088316BC0083120C1AD02B8316CB2BA7
:1017A0009900DF0AC02B61080C1ED42B9900322E41
:1017B00030088316BD008A11831205258A15780822
:1017C0008316B900390EBC00F030BC058312310815
:1017D0008316BD008A11831205258A1578088316A1
:1017E0003C07B90083128D119413831611148312D0
:1017F0008D1DFC2B8316F22B941F002C8316F22BCD
:101800008316111C052C8312002C3908BD008A1187
:10181000831216258A1533088316BD008A11831298
:1018200005258A1578088316BA003A0EBC00F030F8
:10183000BC05831234088316BD008A118312052566
:101840008A15780883163C07BA003A08BD008A1149
:10185000831216258A1536088316BD008A11831255
:1018600005258A1578088316BA003A0EBC00F030B8
:10187000BC05831237088316BD008A118312052523
:101880008A15780883163C07BA0083128C118316D8
:1018900091149118492C01303907BC00BD008A1100
:1018A000831216258A1572300C1E542C990083164B
:1018B0003A08013C0318792C0130F7008A11831291
:1018C00028258A1578088316BB002C3083120C1A41
:1018D0006B2C8316662C990083163B08BC00BD0157
:1018E0008A118312C0248A158316BA038312572CD7
:1018F0008316F7018A11831228258A157808831622
:10190000BB002C3083120C1A872C8316822C990072
:1019100083163B08BC00BD018A118312C0248A15BE
:10192000831611151119922C0D3083120C1A9A2C52
:101930008316952C99000A300C1E9C2C9900322E8F
:101940008C1EA02C1A08AE008C1EA42C1A08AF0006
:101950002F08E40018302E07E5002E088316BD007E
:1019600083122F088316BC001E30FA00FE3083124B
:1019700003178D007A088F00831603133C08831227
:1019800003178C00831603133D08831203178E0080
:1019900083168C170C15831203130B08F8008B1396
:1019A0008316031755308D00AA308D008C1400006B
:1019B00000008C18D92C0C117808831203138B04A7
:1019C000E101C41273300C1EE32C9900322E7430E6
:1019D0000C1EE82C99002C300C1EEC2C99004508AC
:1019E0008316BC00BD018A118312C0248A150D30F4
:1019F0000C1EF82C99000A300C1EFC2C9900322E7B
:101A00008C1E002D1A08AE008C1E042D1A08AF0083
:101A10002F08E40018302E07E50065081D3C031868
:101A20001C2DFF3A031D182D6408FE3C03181C2DC5
:101A30001E30E500FE30E40044121830E300E201FD
:101A400063086502031C6F2D031D2A2D64086202C2
:101A500003186F2D441A2E2D88122F2D88168C1ED8
:101A60002F2D1A08DF008316BD0183125F0883162D
:101A7000BC0083126308FA00620803178D007A081D
:101A80008F00831603133C08831203178C00831600
:101A900003133D08831203178E0083168C170C1551
:101AA000831203130B08F8008B13831603175530AA
:101AB0008D00AA308D008C14000000008C185E2D63
:101AC0000C117808831203138B041030C4065F08CE
:101AD0000C1E682D9900E20A0319E30A202D8812D2
:101AE000FF30E500E40075300C1E742D9900322E95
:101AF00030088316BD008A11831205258A157808DF
:101B00008316BA003A0EBC00F030BC0583123108CF
:101B10008316BD008A11831205258A15780883165D
:101B20003C07BA0083128D1194138316111483128B
:101B30008D1D9C2D8316922D941FA02D8316922D02
:101B40008316111CA52D8312A02D3A08BD008A1101
:101B5000831216258A1533088316BD008A11831255
:101B600005258A1578088316BA003A0EBC00F030B5
:101B7000BC05831234088316BD008A118312052523
:101B80008A15780883163C07BA003A08BD008A1106
:101B9000831216258A1536088316BD008A11831212
:101BA00005258A1578088316BA003A0EBC00F03075
:101BB000BC05831237088316BD008A1183120525E0
:101BC0008A15780883163C07BA003A08BD008A11C6
:101BD000831216258A15831611151119ED2D7730EC
:101BE00083120C1AF52D8316F02D99000D300C1E62
:101BF000F72D99000A300C1EFB2D9900322EFF3074
:101C0000E500E40008130516AA01AB0108127830BC
:101C10000C1E082E9900322E7A300C1E0D2E9900C3
:101C20000D300C1E112E99000A300C1E152E990035
:101C30008A010028322E8316BC013C088A118312C7
:101C4000DC208A158316BC0AF70083120C1A2A2E90
:101C50008316252E9900143083163C02031D1D2E79
:101C60008312322EC2018C128A110A122D2848309A
:0C1C70006C07840083130008F8000034A7
:10200000EC01ED016D080A12F5200A16ED0AF70041
:1020100077080C1E092899001B306D02031D022849
:10202000291429088316870000308312071801300D
:10203000F700770DED00ED0DED0DF830ED05A9146D
:102040002908831687000030831287180130F700B3
:10205000F70DF70DFC30F70577086D07EE00291531
:102060002908831687000030831207190130F70012
:102070000310F70D77086E07EF00A91629088316DD
:10208000870000308312871A01306F07EC006C085C
:10209000F70001307702031956280230770203193E
:1020A000582A043077020319DE2A202B8316A30155
:1020B0000A12831218260A168316A3010A12831223
:1020C00023260A168316A3010A1283122E260A1645
:1020D0008316A3010A12831239260A168316A30156
:1020E0000A12831264260A1601308316A3000A120C
:1020F000831264260A1602308316A3000A12831282
:1021000099270A167808ED0004308316A3000A12F6
:10211000831299270A167808EE0005308316A3006B
:102120000A12831299270A167808EF0001308316E5
:10213000A3000A12831299270A167808F000831662
:10214000A3010A12831299270A167808F1006D0874
:10215000143C031CAD280030AE2801308316A200C9
:102160007108143C031CB6280030B7280130220542
:10217000A3007008143C031CBF280030C0280130A5
:102180002305003A0319CB280130A3000A12831259
:10219000A2270A168316760883126D02003A031DE1
:1021A000D3280030D42801308316A3007608831288
:1021B0006D028316A400053C031CE0280030E128D2
:1021C00001302305A50083126D08103C031CEA288A
:1021D0000030EB28013083162505003A0319F22858
:1021E0007E14F3287E10720883126E02003A031DDB
:1021F000FB280030FC2801308316A30072088312EC
:102200006E028316A400053C031C0829003009292E
:1022100001302305A50083126E08103C031C12290F
:1022200000301329013083162505003A03191A29B5
:10223000FE141B29FE10730883126F02003A031D5F
:1022400023290030242901308316A3007308831248
:102250006F028316A400053C031C3029003031298D
:1022600001302305A50083126F08103C031C3A2996
:1022700000303B29013083162505003A0319422915
:102280007E1543297E1175087102003A031D4A2903
:1022900000304B290130A30075087102A400053CF1
:1022A000031C54290030552901302305A50071086D
:1022B000103C031C5D2900305E2901302505003AE1
:1022C00003196429FE156529FE1174087002003A8D
:1022D000031D6C2900306D290130A30074087002C1
:1022E000A400053C031C7629003077290130230522
:1022F000A5007008103C031C7F29003080290130A4
:102300002505003A031986297E1687297E1200309A
:102310007E180130A2000530AA002208AB000A1284
:102320008312AD270A167808053C8316A3000030F7
:10233000FE190130A4000A30AA002408AB000A12DA
:102340008312AD270A16780883162302A5000030F1
:10235000FE180130F7000310F70D77082507A600D7
:1023600000307E190130F700F70DF70DFC30F7054E
:1023700077082602A70000307E1A0130A800063038
:10238000AA002808AB000A128312AD270A167808A3
:1023900083162707FC0000307E180130A2000530AC
:1023A000AA002208AB000A128312AD270A16780889
:1023B000053C8316A3000030FE190130A40006304E
:1023C000AA002408AB000A128312AD270A16780867
:1023D00083162307A5000030FE180130F700F70D23
:1023E000F70DFC30F70577082502A60000307E19AE
:1023F0000130F7000310F70D77082607A70000301B
:102400007E1A0130A8000A30AA002808AB000A1280
:102410008312AD270A16780883162702FD007C0276
:102420000319292A7D08803AF7007C08803A770250
:102430000318222A0130A3000A128312D4270A1695
:10244000282A83160130A3000A128312DF270A16F6
:1024500083167C08A3007D08A4000A128312EA27D1
:102460000A1628308316A3002308A5000A12831237
:1024700050260A168316A3010A128312D4270A16BD
:102480008316A3010A128312DF270A168316A301FB
:102490000A128312A2270A167008F4007108F500C8
:1024A0006E08F2006F08F3006D08F6006E28202B0E
:1024B0008316A3010A12831218260A168316A30193
:1024C0000A12831223260A168316A3010A12831204
:1024D0002E260A168316A3010A12831239260A161B
:1024E00002308316A3000A12831264260A160630ED
:1024F0008316A3000A12831299270A160310780C78
:10250000EE0007308316A3000A12831299270A16D9
:102510000310780C6E07E70002308316A3000A123E
:10252000831264260A1606308316A3000A12831249
:1025300099270A160310780CEE0007308316A300C3
:102540000A12831299270A160310780C6E07E60008
:102550000230670766020319C62A031CC62A033025
:102560008316A3000730A4000A128312EA270A1672
:102570008316A3010A128312D4270A160130831688
:10258000A3000A128312DF270A16DC2A07308316FB
:10259000A3000330A4000A128312EA270A160130AE
:1025A0008316A3000A128312D4270A168316A301E6
:1025B0000A128312DF270A168C2A202B8316A30106
:1025C0000A12831218260A168316A3010A1283120E
:1025D00023260A168316A3010A1283122E260A1630
:1025E0008316A3010A12831239260A160A308316AB
:1025F000A3000530A4000A128312EA270A16043049
:10260000ED00E1308316A5000A12831250260A1647
:10261000ED0B012BFB308316A300F630A4000A1249
:102620008312EA270A160430ED00E1308316A50074
:102630000A12831250260A16ED0B152BF62A202BB0
:102640008A110A16AE2B840183131F3083050630CE
:1026500083169F000A30990026309800903083122C
:102660009800FF30A900A915290883168700831256
:1026700029162908831687003130930028308312E9
:1026800094008316941714138312AA01AB01AC01B2
:102690002D14AD142D15AD152D12AD12C2012D1333
:1026A000AD134310C3104311C3114312C31243139C
:1026B000C3134410C4104411C411C501C601C7019D
:1026C000DC01DD01E601E7018F018E010A12372DE1
:1026D0000A16A91429088316870000308312871868
:1026E0000130003A031DAD2B2915290883168700F8
:1026F0000030831207190130003A031DAD2BA916D3
:1027000029088316870000308312871A0130003AA7
:10271000031DAD2B2914290883168700003083126E
:1027200007180130003A031D992BFF30E500E40043
:10273000AC2BFE3003178D001E308F0083168C17D4
:102740000C140000000083120E08FA000C0803139A
:10275000E40018307A07E500AE2B002883168C12AF
:102760008312640FB62B650FB62B8E2E0030C41A61
:102770000130003A031DD52B0F08FA000E08F700B0
:102780000F087A02031DBC2B7708ED007A08EE00D3
:102790006E087C3C0318D52BFF3A031DD32B6D0824
:1027A000003C0318D52BC416ED2B0030C41A0130A1
:1027B000013C031DED2B0F08FA000E08F7000F086F
:1027C0007A02031DDB2B7708ED007A08EE006E0815
:1027D0007C3C031CED2BE10AC412EC010A12F32F1E
:1027E0000A166508E3006408E200E901EA016B10DB
:1027F000EB106B11620803178D00031363080317B6
:102800008F0083168C170C140000000083120E0832
:10281000FA000313ED0103170C080313EC00FC3E50
:1028200003187D2C043E9E2EE20A0319E30A620877
:1028300003178D000313630803178F0083168C178B
:102840000C140000000083120313ED0103170C08A1
:102850000313EC00E9007D2CE20A0319E30A620885
:1028600003178D000313630803178F0083168C175B
:102870000C140000000083120313ED0103170C0871
:102880000313EC00EA007D2CE20A0319E30A620854
:1028900003178D000313630803178F0083168C172B
:1028A0000C140000000083120313ED0103170C0841
:1028B0000313EC00E800681C5E2C6B14E81C612C10
:1028C000EB147D2CE20A0319E30A620803178D005A
:1028D0000313630803178F0083168C170C14000072
:1028E000000083120313ED0103170C080313EC001F
:1028F000E800680B7C2C6B157D2CE20A0319E30AB7
:10290000620803178D000313630803178F008316F3
:102910008C170C140000000083120E08FA00031339
:10292000ED0103170C080313EC00FF3C031DFA2B09
:1029300069088316A30083126A088316A4000A128A
:102940008312EA270A1600306B190130EC00831657
:10295000A3000A128312A2270A1600306B18013056
:10296000EC008316A3000A128312D4270A16003043
:10297000EB180130EC008316A3000A128312DF2744
:102980000A16E20A0319E30A620803178D0003130B
:10299000630803178F0083168C170C1400000000C7
:1029A00083120E08FA000313ED0103170C0803133A
:1029B000EC00FF3C03198E2E4416620803178D00AD
:1029C0000313630803178F0083168C170C14000081
:1029D000000083120313ED0103170C080313EC002E
:1029E000DE005E0FF42C502E5E08F70004307702F4
:1029F00003197F2D0530770203197F2D06307702EA
:102A000003197F2D0730770203197F2D08307702D5
:102A100003197F2D0930770203197F2D0A307702C1
:102A200003197F2D0B30770203197F2D0C307702AD
:102A30000319A82D0D3077020319A82D0E30770247
:102A40000319A82D0F3077020319A82D1030770233
:102A50000319A82D113077020319A82D123077021F
:102A60000319A82D133077020319A82D143077020B
:102A70000319D12D153077020319EE2D843077021A
:102A80000319F22D853077020319F22D8630770273
:102A90000319F22D873077020319F22D883077025F
:102AA0000319F22D893077020319F22D8A3077024B
:102AB0000319F22D8B3077020319F22D8C30770237
:102AC00003191F2E8D30770203191F2E8E307702C7
:102AD00003191F2E8F30770203191F2E90307702B3
:102AE00003191F2E9130770203191F2E923077029F
:102AF00003191F2E9330770203191F2E4C2EE20A62
:102B00000319E30A04305E02E00060088316A300A4
:102B10000A12831299270A167808EC006208031734
:102B20008D000313630803178F0083168C170C1492
:102B30000000000083120E08FA000313EE010317D1
:102B40000C080313ED006C02031CA72D44124C2E3D
:102B5000E20A0319E30A0C305E02E0006008EC00B0
:102B60000A128A1537260A168A117808EC006208BC
:102B700003178D000313630803178F0083168C1748
:102B80000C140000000083120E08FA000313EE017B
:102B900003170C080313ED006C02031CD02D441224
:102BA0004C2EE20A0319E30A620803178D0003138F
:102BB000630803178F0083168C170C1400000000A5
:102BC00083120E08FA000313ED0103170C08031318
:102BD000EC0061020318ED2D44124C2EE20A031999
:102BE000E30A4C2EE20A0319E30A5E087F39E0008B
:102BF0000430E00260088316A3000A1283129927AA
:102C00000A167808EC00620803178D0003136308A6
:102C100003178F0083168C170C140000000083121A
:102C20000E08FA000313EE0103170C080313ED005E
:102C30006C0203191D2E03181E2E44124C2EE20A9C
:102C40000319E30A5E087F39E0000C30E0026008F7
:102C5000EC000A128A1537260A168A117808EC0049
:102C6000620803178D000313630803178F00831690
:102C70008C170C140000000083120E08FA000313D6
:102C8000EE0103170C080313ED006C0203194A2E22
:102C900003184B2E44124C2EE20A0319E30ADD2CD2
:102CA000E20A0319E30A441E892E620803178D0005
:102CB0000313630803178F0083168C170C1400008E
:102CC000000083120313ED0103170C080313EC003B
:102CD00001306207EE006308EF000318EF0A6E0888
:102CE00003178D0003136F0803178F0083168C17CB
:102CF0000C14000000008312F0010C080313EF0015
:102D00006F08E40018306C07E5008F018E01E101C7
:102D1000C4120230E2070318E30AC42C83168C168F
:102D200002308312EC00F7308316A6000A128312D9
:102D300044260A16EC0B932EAE2B63000A108A145D
:0C2D40000A158207142C2C2C442C622C49
:02400E003A3D39
:00000001FF
